:100000000C9492060C94BA060C94BA060C94BA0698
:100010000C94BA060C94BA060C94BA060C94BA0660
:100020000C94BA060C94BA060C94160C0C94850C1D
:100030000C94BA060C94BA060C94BA060C94BA0640
:100040000C94BA060C94BA060C94BA060C94BA0630
:100050000C94BA060C94BA060C94BA060C94B70E1B
:100060000C94BA060C94BA060C94BA060C94BA0610
:100070000C94BA060C94BA060C94BA060C94BA0600
:100080000C94010F0C94BA060C94BA060C94BA06A0
:100090000C94BA060C94BA060C94BA060C94BA06E0
:1000A0000C94BA060C94BA060C94BA060000000030
:1000B000003E5B4F5B3E3E6B4F6B3E1C3E7C3E1CEE
:1000C000183C7E3C181C577D571C1C5E7F5E1C0034
:1000D000183C1800FFE7C3E7FF0018241800FFE7EB
:1000E000DBE7FF30483A060E2629792926407F05AE
:1000F0000507407F05253F5A3CE73C5A7F3E1C1CC4
:1001000008081C1C3E7F14227F22145F5F005F5F83
:1001100006097F017F006689956A6060606060946F
:10012000A2FFA29408047E040810207E2010080874
:100130002A1C08081C2A08081E101010100C1E0C7F
:100140001E0C30383E3830060E3E0E060000000011
:100150000000005F00000007000700147F147F14F8
:10016000242A7F2A1223130864623649562050003D
:1001700008070300001C2241000041221C002A1C29
:100180007F1C2A08083E0808008070300008080814
:100190000808000060600020100804023E51494534
:1001A0003E00427F400072494949462141494D3352
:1001B0001814127F1027454545393C4A49493141B9
:1001C000211109073649494936464949291E000087
:1001D00014000000403400000008142241141414DC
:1001E0001414004122140802015909063E415D59C8
:1001F0004E7C1211127C7F494949363E41414122D1
:100200007F4141413E7F494949417F090909013EFA
:10021000414151737F0808087F00417F4100204021
:10022000413F017F081422417F404040407F021C33
:10023000027F7F0408107F3E4141413E7F0909094A
:10024000063E4151215E7F09192946264949493216
:1002500003017F01033F4040403F1F2040201F3FDC
:100260004038403F63140814630304780403615961
:10027000494D43007F4141410204081020004141A3
:10028000417F04020102044040404040000307084F
:100290000020545478407F2844443838444444284B
:1002A000384444287F385454541800087E090218F2
:1002B000A4A49C787F0804047800447D400020407A
:1002C000403D007F1028440000417F40007C0478BE
:1002D00004787C080404783844444438FC18242406
:1002E0001818242418FC7C08040408485454542486
:1002F00004043F44243C4040207C1C2040201C3C03
:100300004030403C44281028444C9090907C4464F9
:10031000544C44000836410000007700000041368C
:10032000080002010204023C2623263C1EA1A16112
:10033000123A4040207A3854545559215555794144
:100340002154547841215554784020545579400C1B
:100350001E527212395555555939545454593955FC
:100360005454580000457C410002457D420001453F
:100370007C40F0292429F0F0282528F07C545545AC
:10038000002054547C547C0A097F4932494949323F
:100390003248484832324A4848303A4141217A3A54
:1003A00042402078009DA0A07D39444444393D401E
:1003B00040403D3C24FF2424487E4943662B2FFCCB
:1003C0002F2BFF0929F620C0887E09032054547979
:1003D000410000447D413048484A32384040227A4A
:1003E000007A0A0A727D0D19317D2629292F2826C7
:1003F0002929292630484D402038080808080808CF
:100400000808382F10C8ACBA2F102834FA00007B27
:10041000000008142A142222142A1408950022002D
:1004200095AA005500AAAA55AA55AA000000FF00E7
:10043000101010FF00141414FF001010FF00FF1024
:1004400010F010F0141414FC001414F700FF000056
:10045000FF00FF1414F404FC141417101F10101FD5
:10046000101F1414141F00101010F0000000001FC3
:10047000101010101F10101010F010000000FF10CE
:100480001010101010101010FF10000000FF1400CA
:1004900000FF00FF00001F10170000FC04F41414FC
:1004A0001710171414F404F40000FF00F7141414C8
:1004B00014141414F700F7141414171410101F1048
:1004C0001F141414F4141010F010F000001F101F6B
:1004D0000000001F14000000FC140000F010F010D9
:1004E00010FF10FF141414FF141010101F00000050
:1004F00000F010FFFFFFFFFFF0F0F0F0F0FFFFFF54
:100500000000000000FFFF0F0F0F0F0F38444438AA
:10051000447C2A2A3E147E02020606027E027E02E5
:1005200063554941633844443C04407E201E200604
:10053000027E020299A5E7A5991C2A492A1C4C7241
:1005400001724C304A4D4D303048784830BC625AC8
:10055000463D3E494949007E0101017E2A2A2A2A58
:100560002A44445F444440514A444040444A514034
:100570000000FF0103E080FF000008086B6B0836F5
:1005800012362436060F090F060000181800000066
:100590001010003040FF0101001F01011E00191D55
:1005A0001712003C3C3C3C0000000000F0F89C8E20
:1005B0008783878E9CF8F00000FEFF03030303038C
:1005C000070EFCF80000FEFF0303030303070EFC05
:1005D000F80000FFFF00000000000000FFFF000027
:1005E000FEFF8383838383C7EE7C380000F8FC0E14
:1005F00007030303070EFCF800003F7FE0C0808084
:10060000C0E07F3FFFFF01010101010101FFFF0089
:1006100000FFFF0C0C0C0C1C3E77E3C100007FFFB9
:10062000C0C0C0C0C0E0703F1F00001F3F70E0C0EE
:10063000C0C0E0703F1F00007FFFC1C1C1C1C1E366
:10064000773E1C00001F3F70E0C0C0C0E0703F1F3D
:10065000000000000001FFFF01000000D5F08D1434
:10066000A1C881CFD9F1AF200008249F42C24282A5
:100670000207001998A5A56E0000003B1013121187
:100680001018009C48484848488C000102020202A9
:1006900002010008249F42C242820207001998A565
:1006A000A56E0000003B1013121110180006081C64
:1006B0001212120C00000000000000000008249F2D
:1006C00042C242820207001998A5A56E0000003BB5
:1006D000101312111018000C12120C12120C000040
:1006E0000000000000000008249F42C2428202076E
:1006F000001998A5A56E0000003B101312111018E8
:10070000000404080808101C00000000000000009D
:100710000008249F42C242820207001998A5A56ED4
:100720000000003B101312111018000C1212120ED0
:10073000041800000000000000000008249F42C2CE
:1007400042820207001998A5A56E0000003B101315
:1007500012111018000E1010100C041800000000E8
:10076000000000000008249F42C2428202070019D4
:1007700098A5A56E0000003B101312111018000878
:10078000081E0A0C0C080000000000000000000811
:10079000249F42C242820207001998A5A56E00005C
:1007A000003B101312111018000E10100C08100E40
:1007B00000000000000000000008249F42C24282A6
:1007C0000207001998A5A56E0000003B1013121136
:1007D0001018001E14081010120C00000000000079
:1007E00000000008249F42C242820207001998A517
:1007F000A56E0000003B101312111018001C080811
:100800000808080C0000000000000000000840007C
:1008100000000000000000389090A82844CE00E3BB
:10082000949494DB000000616070F0D090980046D2
:10083000464E4F4B49590022323A3E2E262200495D
:10084000000049494949000000000000000000087C
:1008500040000000000080C0006792929565081972
:10086000003C1212121B0000008E42222222428201
:1008700000E70C88E8682CE700780909390808784F
:1008800000490000494949490000000000000000FB
:100890000064003200640032004B0032004B003232
:1008A0000032003200320032000080804000000040
:1008B0000000000000000000000000000000000038
:1008C0000000E02020207020000000000000E04038
:1008D000C0404040E00000000000000000000000B8
:1008E0000000000000000000000000000000000008
:1008F00000000000000000000000000000000000F8
:1009000000000000000000000000000000000000E7
:10091000000000E0808080808080808888F800006F
:1009200000000000000000000000000000000000C7
:1009300000000000000000000000000000000000B7
:1009400000000609090906000000000000009C489C
:10095000C94ABE02010000000000000000000000C3
:100960000000000000000000000000000000000087
:10097000000000000000000000000000000000E097
:10098000101010101030D0101018100000000000CF
:10099000000000C3201010101020C008080F000035
:1009A0000000000000000000000000000000000047
:1009B00000000030A09030000000000000000000A7
:1009C0000000739413913E10000000000000CD1051
:1009D000CD4598000000000000000000000000006D
:1009E00000000000000000E0101020F010E02010D7
:1009F0001020C0000000000000000000000000E027
:100A00001112121212111800000000000000000064
:100A10000000008182444444242271000000000050
:100A200000000000000000000000000000000000C6
:100A30000000007348487300000000000000000040
:100A40000000DF4A4B4AFD4000000000000070A19A
:100A5000E0A02120300000000000000000000000A5
:100A6000000000000000000102040473901021C285
:100A70001217E000000000000000000000000072FB
:100A80002722222222322300000020000000000042
:100A9000000000080815151522227700000000004C
:100AA0000000000000000000000000000000000046
:100AB000000000B9A5A5B901010000000000000078
:100AC0000000250000000000000000006080998404
:100AD0009C546900000000000000000000000000BD
:100AE00000000000000000000000009F0909090943
:100AF000091DE80000000000000000000000000EDA
:100B000084444444448404040406040000000000B7
:100B10000000009C2201013F21A21C0000000000F7
:100B200000000000000000000000000000000000C5
:100B3000000000CA2222C1000000000000000000E6
:100B40000000010000000000000000000000E04183
:100B5000C18286800000000000000000000000004C
:100B6000000000000000000000000073212121218E
:100B700021231C0000000000000000000000000B0A
:100B80009C4848C8488C0B08080C0800000000006E
:100B90000000000301010101011B0D000000000025
:100BA0000000000000000000000000000000000045
:100BB0000000004C5252CC00000000000000000079
:100BC00000000000000000000000000000000C0415
:100BD0000702020201000000000000000000000007
:100BE00000000000000000000000001C2201013F86
:100BF00021221C000000000000000000000000E7AF
:100C00004840404F48E84700000000000000000056
:100C100000000000000000000000000000000000D4
:100C200000000000000000000000000000000000C4
:100C300000000005050503000000000000000000A2
:100C400000000000000000000000000000000000A4
:100C50000000000000000000000000000000000094
:100C60000000000000000000000000000000000084
:100C70000000000000000000000000000000000074
:100C8000000000000006030000000000000000005B
:100C90000000000000000000000000000000000054
:100CA00000000000000000000000000000080B0031
:100CB00002020200000904000001020200000524F3
:100CC0000010010524010101042402060524060088
:100CD000010705810310004009040100020A000019
:100CE00000070502024000000705830240000004DF
:100CF00003090412010002EF020140412336800083
:100D0000010102030141726475696E6F204C4C430E
:100D10000041726475696E6F204C656F6E6172641C
:100D20006F00DA0F11241FBECFEFDAE0DEBFCDBFB8
:100D300012E0A0E0B1E0E0E5F9E202C005900D921A
:100D4000A234B107D9F727E0A2E4B2E001C01D92B6
:100D5000A132B207E1F716E0C2E9D6E004C021975C
:100D6000FE010E949B14C139D107C9F70E941B10D4
:100D70000C94A6140C940000809154020895EAEAA1
:100D8000F2E0A0E0B8E000800EBC8111012C1197C8
:100D9000A0FDFDCF0192B9F70DB408956F927F9237
:100DA0008F929F92AF92BF92CF92DF92EF92FF927B
:100DB0000F931F93CF93DF939C01FA019490319688
:100DC000E491C92CD12CD601A80FB91F109709F4B2
:100DD00075C0CB018E0F911D892B09F46FC0862F32
:100DE0008770F3E075956795FA95E1F7862EA03840
:100DF000B1051CF090E8992E921A91E0FE2FF77041
:100E000009F490E0E695E695E6959E0FFB01E90F63
:100E1000F11D399714F098E0961B4E5F5F4FEB0180
:100E2000D695DC2FCC27D795C795C20FD31FA82EF8
:100E3000082E000CBB08AFEFB0E0082E02C0AA0FCE
:100E4000BB1F0A94E2F7A095B0957B2E282D261B98
:100E50002917A0F58E0106551D4FF12CE12CE91440
:100E600038F5FA01EE0DFF1D249130E00A2C02C086
:100E7000220F331F0A94E2F787FC08C0F801608054
:100E8000E62DEA236E2E622AF8016082882351F053
:100E9000F6E0F8153CF0F801E058FF4F20812721DB
:100EA000232B20832FEFE21AF20A0F5F1F4FD7CFB9
:100EB0004C0D5D1DC058DF4F8394C8CFDF91CF919B
:100EC0001F910F91FF90EF90DF90CF90BF90AF9068
:100ED0009F908F907F906F9008958091140783FD6D
:100EE00006C08091130783FB882780F9089580E06E
:100EF0000895FC018091A902882311F13FB7F8946D
:100F000082E08093E9002091F200822F90E0181691
:100F1000190614F481E090E0882339F0289844E61B
:100F20004093A8024091F1004083222339F02091A0
:100F3000F200211103C02BE62093E8003FBF089583
:100F40008FEF9FEF08952FB7F89483E08093E90027
:100F50009091E800892F807295FF04C09091F20073
:100F600080E4891B2FBF08958091A00281110DC0DC
:100F700082E080939C0284E080939D0210929F0205
:100F800010929E0281E08093A0028CE992E0089585
:100F9000CF93DF931F92CDB7DEB76983DC01ED916C
:100FA000FC910280F381E02D41E050E0BE016F5FD3
:100FB0007F4F09950F90DF91CF91089583E0809343
:100FC000E9008091F200882319F08AE38093E80019
:100FD00008950E94A30790E00895CF93DF931F9296
:100FE000CDB7DEB7FC018485958597FD08C02FEF4E
:100FF0003FEF358724870F90DF91CF910895CE0181
:1010000001960E947907019719F4898190E0F3CF46
:101010008FEF9FEFF0CF0F931F93CF93DF931F922C
:10102000CDB7DEB78C01FC018485958597FF0BC099
:10103000CE0101960E947907019771F4898190E0B1
:10104000F80195878487F801848595850F90DF9155
:10105000CF911F910F9108958FEF9FEFF1CFFC017A
:101060008485958597FD0BC09FB7F89482E08093A7
:10107000E9008091F2009FBF90E0019608959FB72C
:10108000F89482E08093E9008091F2009FBF90E0A5
:1010900008954091960250919702209194023091C8
:1010A000950242175307B4F49091E8009570E1F36C
:1010B0009091E80092FD19C08093F1008091960212
:1010C0009091970201968F739927892B19F48EEFCF
:1010D0008093E800809196029091970201969093F8
:1010E00097028093960281E0089580E00895DF9250
:1010F000EF92FF920F931F93CF93DF93D82E8A0125
:10110000EB017B01E40EF51ECE15DF0559F0D7FE8D
:1011100012C0FE0184910E94490821968111F4CFEA
:101120000FEF1FEFC801DF91CF911F910F91FF903B
:10113000EF90DF9008958881EECF0F931F93CF93A8
:10114000DF931F92CDB7DEB782E0898342E450E09F
:101150006DEA7CE080E80E9477080E94B407DC0119
:1011600012960D911C910115110589F0D801ED9190
:10117000FC910280F381E02DBE016F5F7F4FC801BB
:10118000099597FD04C0F80100851185ECCF898190
:101190000F90DF91CF911F910F910895615030F022
:1011A0002091F100FC0120830196F8CF289884E675
:1011B0008093A8020895AF92BF92CF92DF92EF92F0
:1011C000FF920F931F93CF93DF936C017B018B01F1
:1011D000040F151FEB015E01AE18BF08C017D10741
:1011E00059F06991D601ED91FC910190F081E02DCB
:1011F000C6010995892B79F7C501DF91CF911F9120
:101200000F91FF90EF90DF90CF90BF90AF90089537
:101210003FB7F8948091500290915102A0915202F0
:10122000B091530226B5A89B05C02F3F19F0019637
:10123000A11DB11D3FBFBA2FA92F982F8827BC0130
:10124000CD01620F711D811D911D42E0660F771F58
:10125000881F991F4A95D1F708958F929F92AF9258
:10126000BF92CF92DF92EF92FF926B017C010E94BE
:1012700008094B015C01C114D104E104F104B9F087
:101280000E940809681979098A099B09683E734018
:101290008105910580F321E0C21AD108E108F10827
:1012A00088EE880E83E0981EA11CB11CE4CFFF904D
:1012B000EF90DF90CF90BF90AF909F908F90089568
:1012C0008F929F92AF92BF92CF92DF92EF92FF9256
:1012D0000F931F93CF93DF936C017B018A01809161
:1012E0000F01882309F45CC08091A902882309F4C6
:1012F00057C080919B0280FF05C08091E000826012
:101300008093E000E801B12C8AEFA82E93E0892EAB
:101310002AE3922E209711F4BB20D9F10E94A30753
:1013200081110AC0AA94AA20D9F161E070E080E09E
:1013300090E00E942D09EECF8C171D0611F00CF0E5
:101340008C2F9FB7F8948092E9002091E80025FD4A
:1013500002C09FBFDFCF282F30E0C21BD30BF701A5
:10136000815020F041914093F100FACFE20EF31E3C
:10137000BB2021F09092E800B12CEBCF8091E800E7
:1013800085FDE7CF9092E800BB24B394209709F342
:10139000F3CF5D9884E680939A02101611063CF014
:1013A00081E090E0F6019383828310E000E0C801C1
:1013B000DF91CF911F910F91FF90EF90DF90CF9031
:1013C000BF90AF909F908F90089520915902E09127
:1013D0005702F0915802CF010296909358028093E1
:1013E0005702222319F0859194910895808191816B
:1013F0000895CF92DF92EF92FF92CF93DF930E94F6
:10140000E509811520E8920791F4809171008D7FA4
:101410008093710010929100469847981092440270
:10142000DF91CF91FF90EF90DF90CF90089521E072
:1014300020934402813020E8920751F480915502B4
:101440009091560290935802809357020E94E509AA
:1014500097FD05C020914302222309F454C0209136
:101460004202211150C021E020934502EC01DF77B8
:10147000209709F04BC081E08093460246983FE9EF
:10148000C32E3FE0D32EE12CF12CCAEFD0E0E09147
:101490000807F09109070995811103C081E0809345
:1014A000460280914502882329F0809146028823D4
:1014B00009F43FC047980E94E5090097F1F19C01AB
:1014C000DE010E948C14DC01CB0129E0B595A795C3
:1014D000979587952A95D1F7109290002AE020934E
:1014E0009100D0929900C092980080934702909307
:1014F0004802A0934902B0934A0280917100826031
:10150000809371008DCF10924502B0CF9E0150E0C4
:1015100040E060E472E48FE090E00E944B146901C7
:101520007A0181E0C81AD108E108F1081092460258
:10153000AECF4699BFCF479ABECF8FEF9FEFDC016A
:10154000CBCF2D9A0895BC0190E080E00C942D093A
:101550008FB18095807F669B88601C9B8460089516
:101560003E9A3F9A81E080935402089520E191E0F1
:1015700061FD94E060FD990F62FD9295687F269F62
:10158000D0011124A80FA655BD4F8C9140FF03C078
:10159000892B8C93089590958923FBCFAF92BF92AE
:1015A000CF92DF92EF92FF920F931F93CF93DF932F
:1015B0006B01EC015C01A40EB11C7B01E20EF11C7D
:1015C000CA15DB05E4F48601D7FE02C010E000E096
:1015D000C70121E4E216F10414F080E490E008175A
:1015E00019075CF4C038D10528F441E0B801CE01F8
:1015F0000E94B60A0F5F1F4FEBCF2196E1CFDF911C
:10160000CF911F910F91FF90EF90DF90CF90BF90FF
:10161000AF9008952F923F924F925F926F927F9278
:101620008F929F92AF92BF92CF92DF92EF92FF92F2
:101630000F931F93CF93DF93CDB7DEB728970FB6E5
:10164000F894DEBF0FBECDBF9E838D836A3061F5F7
:10165000DC0155968C91B8E08B9F90011124ED81AF
:10166000FE8181899289820F931F928B818B108AD0
:10167000178681E090E028960FB6F894DEBF0FBE83
:10168000CDBFDF91CF911F910F91FF90EF90DF9031
:10169000CF90BF90AF909F908F907F906F905F9012
:1016A0004F903F902F9008956D3019F32D813E811A
:1016B00038872F83D9011F960D911C9150970038C0
:1016C00011050CF07CC05196AD90BC90B0E4AB1607
:1016D000B1040CF074C0F901258825E0C801229EF0
:1016E000800D911D1124181619060CF068C0622C8B
:1016F000712CC30133E0880F991F3A95E1F78A0DE9
:101700009B1D181619060CF05AC0F489FB83AF8193
:10171000B8855396BC91BC83629FB0011124FB0134
:10172000E455FF4F2F011982F2018491F981F530C0
:1017300009F480E0450128E02A83A82FB0E0BE83A9
:10174000AD833C8080FF3B80311004C0BB81EC81C5
:10175000BE17F9F078018E2D801B8215D0F4D12CA4
:10176000C12CC21490F4F0E8EF16F10450F4B60165
:10177000680D791D6034710520F4432DC7010E9466
:10178000B60A2FEFC21AD20AECCF3FEFE31AF30AE0
:10179000E2CF8D819E81959587959A8191509A830C
:1017A000860C971C9111C9CFA981AF5FA983BFEFA8
:1017B0004B1A5B0A060D171DA63009F0B5CFEF8155
:1017C000F8852589422F50E087859089F6E02F9F84
:1017D000800D911D1124AF81B88550969C938E93F6
:1017E0001F9756962C915697222309F442CF6AEF01
:1017F00064039001659F300D112420583F4F281736
:1018000039070CF036CFED91FC9111970190F081E2
:10181000E02D6AE0CD0109952CCF0895089590E060
:1018200080E008950C9435140E94A1141F920F9229
:101830000FB60F9211248F939F938091E1009091A6
:10184000E100937F9093E10083FF0FC01092E900C5
:1018500091E09093EB001092EC0092E39093ED00F6
:101860001092A90298E09093F00082FF22C093E0CA
:101870009093E9009091F200992319F09AE39093E4
:10188000E80090919A02992341F090919A02915028
:1018900090939A02911101C05D9A9091A8029923A8
:1018A00041F09091A80291509093A802911101C02B
:1018B000289A84FF18C08091E2008E7E8160809318
:1018C000E2008091E1008F7E8093E10080919B0295
:1018D0008E7E806180939B029F918F910F900FBEAF
:1018E0000F901F90189580FFF7CF8091E2008E7EB9
:1018F00080618093E2008091E1008E7E8093E10020
:1019000080919B028E7E8160E5CF1F920F920FB671
:101910000F921124CF92DF92EF92FF920F931F93B9
:101920002F933F934F935F936F937F938F939F93E7
:10193000AF93BF93EF93FF93CF93DF93CDB7DEB712
:101940006C97DEBFCDBF1092E9008091E80083FF65
:1019500025C068E0CE0145960E94CE0882EF8093B4
:10196000E8008D8987FF39C09091E80090FFFCCF97
:10197000982F907609F034C19E894F89588D2F8910
:10198000F88C911131C0803861F580919902809373
:10199000F1001092F1008EEF8093E8006C960FB684
:1019A000F894DEBF0FBECDBFDF91CF91FF91EF91D5
:1019B000BF91AF919F918F917F916F915F914F9167
:1019C0003F912F911F910F91FF90EF90DF90CF905B
:1019D0000F900FBE0F901F9018959EEF9093E80008
:1019E000C7CF1092F100D5CF913059F48111D3CFE8
:1019F0004130510581F6809199028D7F8093990243
:101A0000CACF933049F48111C6CF4130510519F640
:101A1000809199028260F2CF953041F48091E80084
:101A200080FFFCCF20682093E300B5CF963009F00B
:101A3000A9C00B8D1C8D22E01092E9001092970234
:101A400010929602F2122EC01092950210929402F9
:101A50000E949D081F8299E09983FA8291E09E83FB
:101A600090EA98879AEF9987209196023091970291
:101A7000275F3F4F3C832B838D831092E9001092A8
:101A8000970210929602109395020093940249E0F7
:101A900050E0BE016F5F7F4F80E00E9477080E9498
:101AA0009D0879CF10939502009394020E94B40789
:101AB000DC0112960D911C910115110509F451C11B
:101AC000D801ED91FC910480F581E02DBE016B5EA3
:101AD0007F4FC8010995009709F03EC1F8010085C4
:101AE0001185EACFF3E0FF120EC08F89882309F435
:101AF00040C0823061F440E860E181E19DE00E94F5
:101B0000620F811148CF81E28093EB0047CF813093
:101B100029F440E86BE085E09DE0F1CF833099F750
:101B20000E94B407DC011296ED90FC908E010F5FCD
:101B30001F4F6801E114F10479F0D701ED91FC9198
:101B40000680F781E02DB801C7010995080F111D26
:101B5000F701E084F184EECFD8011C92F6010190E8
:101B60000020E9F73197BF016C197D0940E0C601FB
:101B7000C6CF6FEE7CE0FB01449150E080E80E940C
:101B8000770809CF973009F4BECF983021F481E06F
:101B90008093F10000CF993009F0FDCE837009F0F9
:101BA000B2CFE5E1F2E081E031E096E3219122233A
:101BB00071F08093E9003093EB00DF0111972C91D5
:101BC0002093EC009093ED008F5F873079F78EE7DC
:101BD0008093EA001092EA008F898093A902DBCEFD
:101BE0008B8D9C8D1092E9001092970210929602B4
:101BF0009093950280939402898D811192C08E8971
:101C00009D89913A49F4813209F07DCF47E050E057
:101C100068E071E080E0B3CF913209F074CF833295
:101C200069F48F89988DB0E0A0E0809304019093CF
:101C30000501A0930601B0930701ADCE803269F48F
:101C40008091E80082FFFCCF67E088E091E00E948D
:101C5000CE088BEF8093E8009ECE823209F09BCEB7
:101C60008F8980930F01EEEFFFE7859194918B3F71
:101C70009C4D51F1E0E0F8E080910801909109015C
:101C8000A0910A01B0910B01803B9440A105B105E0
:101C9000F1F480910F0180FD1AC0EE3F8AE0F80751
:101CA00089F587E797E7918380838091600080932F
:101CB000980288E19BE00FB6F894A89580936000A5
:101CC0000FBE9093600067CEEEEFFAE0D5CF808133
:101CD00091818737974709F05ECEA8958091600083
:101CE0008861809360008091980280936000EE3F4D
:101CF0002AE0F20789F08091FE0A9091FF0A918311
:101D0000808349CE808191818737980751F29093E3
:101D1000FF0A8093FE0AC5CF1092FF0A1092FE0AB6
:101D20003ACE0E94B407DC0112960D911C91011568
:101D3000110509F4E8CED801ED91FC910190F081F4
:101D4000E02DBE016B5E7F4FC8010995811123CE46
:101D5000F80100851185EBCF181619060CF41BCE7F
:101D6000D2CEF1E0FF12BECE63EF7CE004CF1F9233
:101D70000F920FB60F9211242F933F938F939F933F
:101D8000AF93BF9380914C0290914D02A0914E026F
:101D9000B0914F0230914B0223E0230F2D3758F5BD
:101DA0000196A11DB11D20934B0280934C0290938C
:101DB0004D02A0934E02B0934F0280915002909139
:101DC0005102A0915202B09153020196A11DB11D82
:101DD0008093500290935102A0935202B093530209
:101DE000BF91AF919F918F913F912F910F900FBE17
:101DF0000F901F90189526E8230F0296A11DB11D84
:101E0000D2CF1F920F920FB60F9211242F933F93B0
:101E10004F935F936F937F938F939F93AF93BF93F2
:101E2000EF93FF938091470290914802A09149025D
:101E3000B0914A02892B8A2B8B2B09F440C08091E8
:101E4000460281110BC088B190E4892788B980913E
:101E50004502882319F088B1805888B980914702DB
:101E600090914802A0914902B0914A0218161906B1
:101E70001A061B069CF48091470290914802A0919B
:101E80004902B0914A020197A109B1098093470222
:101E900090934802A0934902B0934A02FF91EF91B8
:101EA000BF91AF919F918F917F916F915F914F9172
:101EB0003F912F910F900FBE0F901F9018950E9489
:101EC000F909ECCFEF92FF920F931F93CF93DF931B
:101ED000F82E192FE62E042F81E0860F880F0E941E
:101EE000490883E00E944908CF2DD12FEC0EFD2E2A
:101EF000F11CCE15DF05B9F007FF13C0FE01849178
:101F00000E944908182F80E00E94490881232196E9
:101F10008111EFCFDF91CF911F910F91FF90EF9043
:101F200008958881EDCF81E0F5CF0F931F93CF9374
:101F3000DF938C0181E090E00E94120C80FF32C0A0
:101F40008AE090E00E94120C9FEF980F9E3F50F5A0
:101F500022E330E0D80150963C932E931F9728E35C
:101F600030E052963C932E935197CBE0D0E0D801CD
:101F7000ED91FC910190F081E02D682FC801099549
:101F8000CE010E94120C2196C131D10581F780E06B
:101F90000E94BF0688EE93E0DF91CF911F910F91D1
:101FA0000C94A30ADF91CF911F910F91089504978C
:101FB0000C94950FEAEAF6E01382128288EE93E021
:101FC000A0E0B0E084839583A683B7838FE192E09D
:101FD000918380838FEF9FEF95878487EAE0F7E016
:101FE000138212821186128680E1838710861782FF
:101FF000158681E392E0918380838FE392E095835D
:102000008483108A1786128A118A81E0838B148A4E
:10201000858B168A8CEB96E09093090780930807CE
:1020200080E090E8909307078093060746983E9AD1
:1020300047983F9A0895789484B5826084BD84B5AA
:10204000816084BD85B5826085BD85B5816085BDB3
:1020500080916E00816080936E001092810080916B
:1020600081008260809381008091810081608093F3
:102070008100809180008160809380008091910038
:1020800082608093910080919100816080939100A3
:10209000809190008160809390008091C100846065
:1020A0008093C1008091C10082608093C1008091C3
:1020B000C10081608093C1008091C30081608093E2
:1020C000C3008091C00082608093C0008091C200F4
:1020D00081608093C20080917A00846080937A004E
:1020E00080917A00826080937A0080917A0081608A
:1020F00080937A0080917A00806880937A001092B1
:10210000A9021092990210929B028091D7008160DF
:102110008093D70080EA8093D80089B5806189BD1B
:1021200089B5826089BD09B400FEFDCF61E070E031
:1021300080E090E00E942D098091D8008F7C806122
:102140008093D8008091E000807F8093E0008091B0
:10215000E1008E7E8093E1008DE08093E200559A4D
:10216000209A81EC80937C0085B1806F85B984B121
:10217000877E84B984B1876E84B95E9A5F988AB18C
:10218000806D8AB9769A6E9881B3806F81BB899889
:1021900080B38D7080BB80E58CBD81E08DBD85E016
:1021A00090E00E94A30A5F9A85E090E00E94A30A53
:1021B0005E985C98ECE5F6E084918EBD00000DB46D
:1021C00007FEFDCF319636E0E936F307A9F75C9AB2
:1021D00081E8809364008091650081608093650050
:1021E00080E00E94BF060E94A80A87FF15C05C9885
:1021F00085EA8EBD00000DB407FEFDCF5C9A2E98D7
:102200002F982D988091640080628093640081E013
:1022100083BF889513BEFCCF0E94A80A82FF48C0E6
:102220002D980E94A80A84788438E1F40E94A10ABB
:1022300088EC90E00E94A30A2F9882E090E00E9430
:1022400035148F3F29F06FEF82E090E00E943D143B
:1022500084EF91E00E94A30A2F9A0E94A80A847832
:102260008438D9F30E94A80A84718431E1F40E9471
:10227000A10A88EC90E00E94A30A2E9882E090E0E8
:102280000E943514882329F060E082E090E00E94EB
:102290003D1484EF91E00E94A30A2E9A0E94A80A9E
:1022A00084718431D9F388EC90E00E94A30AB4CF02
:1022B0000E94A10A82E090E00E94120C882309F497
:1022C000BFC00E94B00A81E090E00E94120C482F2B
:1022D0004470742E81FF11C041112E98C0EFDFEFC2
:1022E00008E010E06CE6E62EF12C0E94A80A86FFBA
:1022F000ACC02E9A2F9A0E94A10A82E390E00E941D
:10230000A30A0E94A80A8111F8CF0E94B00A8EE8A1
:10231000682E82E0782E91E9492E98E0592E24E02B
:10232000222E312C0DE0F02EEE24E39480E0EAEA38
:10233000F2E081118FEF0024819381938193819347
:102340000394D1F710921C0710921B0710921A07E2
:102350001092190780911307809314070E94A80A0E
:1023600080931307809102019091030183309105BE
:1023700009F444C10CF0FDC0019709F411C1C090EB
:102380000201D0900301C0919002D091910251E0DE
:10239000C516D10409F42EC21C161D06ECF40AE57C
:1023A00012E0912C812CB12CA12CD8016C911196AA
:1023B0007C91119712962C91261B49E0C4010E9432
:1023C000CE0ABFEFAB1ABB0A0C5F1F4FE9E08E0EBF
:1023D000911CCA15DB054CF7F3E0CF16D10409F0C8
:1023E00009C20091920210919302F09EF001F19EB9
:1023F000F00D1124EC0FFD1FEE0FFF1FE05FFE4FED
:1024000060918E0270918F02208149E04C9FC00143
:102410004D9F900D11240E94CE0A0A30110508F03C
:10242000E9C1F801EA5EFD4E0C949B14F2131114FD
:10243000141417141A141D14201423142614291408
:10244000109254023E983F983ECF772029F0C43036
:10245000D10511F42E9A2F9881E00E94BF069E01AB
:10246000D7FF04C0222733272C1B3D0B27703327AF
:10247000CE01D7FD079653E0959587955A95E1F7DC
:10248000D7FF05C00197D801A21BB30B9D01BC016A
:102490007695762F66277795679566557D4FB0E0E0
:1024A000A0E02801421A530A8F3FEFEF9E070CF479
:1024B0003CC048E550E0FD01EC5FF94F5F014B0186
:1024C000F0E88F0E911C8F3F9807A1F0F501E41BF7
:1024D000F50BE4916701C41AD50AC60ED71EF0E0C9
:1024E0001F01022E01C0220C0A94EAF7F601308087
:1024F0002328208221153105A9F0F501E41BF50BF5
:10250000E4916701C41AD50AC80CD91CF0E01F0178
:10251000042C02C0359427940A94E2F7F601308027
:10252000232820824150510971F60196A85ABF4FC5
:1025300060587F4FA03BB10509F0B6CF80E00E9404
:10254000BF068FE090E00E94A30A2196C931D10511
:1025500009F0CBCE772011F02F9A2D9880E991E0E9
:102560000E94A30A0E94A10A8AE097E00E94950FA8
:10257000C4CE8430910509F432C14DE058E005978E
:1025800009F0FDCE70E060E086E790E00E94CE06A4
:102590000E946D07882309F45FC141E050E029C023
:1025A0004BEA58E070E060E090E080E00E94CE06E8
:1025B0000E946D07C0919002D0919102882309F486
:1025C00019C11092930210929202109291021092ED
:1025D000900210928F0210928E02EAE5F2E01182D0
:1025E00010821382128234966E167F06C1F743E082
:1025F00050E05093030140930201C1CE0E946D0749
:10260000882309F462C080919002909191028E30EB
:1026100091050CF043C0C0918E02D0918F02AC01A5
:10262000440F551F440F551FFA01E65AFD4FD18341
:10263000C0836091920270919302F69ED001F79E42
:10264000B00D1124A80FB91FAA0FBB1FA05FBE4F6A
:102650000D90BC91A02D5D01AC0EBD1EB382A28277
:10266000181619060CF0B5C09C0121503109220F33
:10267000331F220F331F8901065A1D4FD801CD90F9
:10268000DC901197AC14BD040CF051C030920301E2
:1026900020920201118210821382128280917100B5
:1026A0008D7F80937100E0925902509258024092BF
:1026B000570250925602409255020E94F9096CE26C
:1026C00071E080E090E00E942D092091000130919E
:1026D000010180918E0290918F02820F931F90933F
:1026E0008F0280938E024091920250919302F49E49
:1026F000F001F59EF00D112440919002509191024D
:10270000E40FF51FEE0FFF1FE05FFE4F4081518188
:10271000480F591F4134510514F497FF30CE3195BD
:1027200021953109309301012093000128CE1296A2
:102730000D911C910C171D070CF4A8CFCC15DD05CD
:1027400014F4D182C0820A151B052CF4FA01E65A52
:10275000FD4F13830283DA01A65ABD4FF901E65AF1
:10276000FD4F4D915C9111972081318142175307A4
:102770000CF494CF12962D913C91428153814217D3
:1027800053070CF48BCF8C30910519F56930710526
:1027900039F4E5E0F0E0F0930301E09302017ECF2D
:1027A0006F5F7F4F70939302609392021092910239
:1027B0001092900210928F0210928E02EAE5F2E0DF
:1027C000118210821382128234966E167F06C1F730
:1027D00065CF019690939102809390025FCF4FE472
:1027E00058E0D0CE43EE57E06CE070E086E790E032
:1027F0000E94CE0680E00E94BF06CC0FDD1F69E17B
:1028000070E06C1B7D0B072E000C880B990B0E944F
:102810002D0940E050E0452B09F488CD0E940000CE
:1028200081CD49EB57E0E0CF4FE857E0DDCF45E6FB
:1028300057E0DACF4BE357E0D7CF41E157E0D4CFB1
:1028400047EE56E0D1CF4DEB56E0CECF43E956E010
:10285000CBCF49E656E0C8CFC0900201D09003012B
:10286000C0919002D091910297CDF999FECF92BD7F
:1028700081BDF89A992780B50895262FF999FECF42
:102880001FBA92BD81BD20BD0FB6F894FA9AF99A8D
:102890000FBE01960895052E97FB1EF400940E942A
:1028A000621457FD07D00E946A1407FC03D04EF44F
:1028B0000C94621450954095309521953F4F4F4FA1
:1028C0005F4F089590958095709561957F4F8F4FDC
:1028D0009F4F0895A1E21A2EAA1BBB1BFD010DC03C
:1028E000AA1FBB1FEE1FFF1FA217B307E407F507C0
:1028F00020F0A21BB30BE40BF50B661F771F881F9C
:10290000991F1A9469F760957095809590959B0131
:10291000AC01BD01CF010895A29FB001B39FC001DA
:10292000A39F700D811D1124911DB29F700D811DFB
:102930001124911D0895EE0FFF1F0590F491E02DD5
:10294000099481E090E0F8940C94A614F894FFCFD9
:1029500001000100FFFFFFFF00E100000000000098
:102960002800280028002800280028002300230031
:102970002300230023002300230028002800280030
:102980002800230023002300230023001E001E0034
:102990001E001E002800280028002300230023001A
:1029A000230023001E001E001E001E001900280028
:1029B0002800280023002300230023001E001E00FF
:1029C0001E00190019001900280028002800230003
:1029D000230023001E001E001E001900190019000C
:1029E0001400280028002300230023001E001E00DE
:1029F0001E001900190019001400140028002800F6
:102A0000230023001E001E001E00190019001900DB
:102A10001400140014002800280023001E001E00CB
:102A200019001900190014001400140014000F00FC
:102A30002800280023001E001E001900190019009C
:102A40001400140014000F000F00280028002300B9
:102A50001E0019001400140014000F000F000A00DB
:102A60000A00050000C1808100000000000000C8CD
:102A7000076009E907DE072F08ED070B08000000D3
:102A8000000A0BDB080F0C0E0C950FFCFF0000D7A3
:022A90000F0035
:00000001FF
